:1007E000003700000004000004D2000000000000F8
:1007F00000000000000000000000000000000000F9
:100800000221FB1211CC22D2AF320002202FD2AF34
:10081000320000022A15022B940000020807000093
:10082000000000021642000000000002080EEF8DDA
:10083000F0A4A8F0CF8CF0A428CE8DF0A42EFE2238
:10084000C2D5EC30E709B2D5E4C39DFDE49CFCEED3
:1008500030E715B2D5E4C39FFFE49EFE120B3CC304
:10086000E49DFDE49CFC8003120B3C30D507C3E4FF
:100870009FFFE49EFE22C5F0F8A3E028F0C5F0F843
:10088000E582158270021583E038F022BB010A89E7
:10089000828A83E0F5F0A3E022500687F009E71989
:1008A00022BBFE07E3F5F009E3192289828A83E47B
:1008B00093F5F074019322BB010A89828A83F0E5E3
:1008C000F0A3F0225006F709A7F01922BBFE06F3A9
:1008D000E5F009F31922E88FF0A4CC8BF0A42CFCEE
:1008E000E98EF0A42CFC8AF0EDA42CFCEA8EF0A496
:1008F000CDA8F08BF0A42DCC3825F0FDE98FF0A425
:100900002CCD35F0FCEB8EF0A4FEA9F0EB8FF0A41B
:10091000CFC5F02ECD39FEE43CFCEAA42DCE35F057
:10092000FDE43CFC2275F008758200EF2FFFEE33EA
:10093000FECD33CDCC33CCC58233C5829BED9AEC52
:1009400099E58298400CF582EE9BFEED9AFDEC99BC
:10095000FC0FD5F0D6E4CEFBE4CDFAE4CCF9A882C6
:1009600022B800C1B90059BA002DEC8BF084CFCE6B
:10097000CDFCE5F0CBF97818EF2FFFEE33FEED3329
:10098000FDEC33FCEB33FB10D703994004EB99FBF0
:100990000FD8E5E4F9FA227818EF2FFFEE33FEEDD9
:1009A00033FDEC33FCC933C910D7059BE99A4007E6
:1009B000EC9BFCE99AF90FD8E0E4C9FAE4CCFB22FD
:1009C00075F010EF2FFFEE33FEED33FDCC33CCC8C6
:1009D00033C810D7079BEC9AE899400AED9BFDECD1
:1009E0009AFCE899F80FD5F0DAE4CDFBE4CCFAE410
:1009F000C8F922EB9FF5F0EA9E42F0E99D42F0EC47
:100A00006480C864809845F022EB9FF5F0EA9E422E
:100A1000F0E99D42F0E89C45F022E8600FECC3133A
:100A2000FCED13FDEE13FEEF13FFD8F122E8600F8B
:100A3000EFC333FFEE33FEED33FDEC33FCD8F12290
:100A4000BB010789828A83020B9D5005E9F8020BDE
:100A500091BBFE05E9F8020BA989828A83020BB5D6
:100A6000BB010789828A83020A9A5005E9F8020BC2
:100A7000FBBBFE05E9F8020AA622BB010789828AB0
:100A800083020BD25005E9F8020BC5BBFE05E9F85D
:100A9000020BDE89828A83020BEBECF0A3EDF0A35C
:100AA000EEF0A3EFF022ECF208EDF208EEF208EF20
:100AB000F222A8828583F0D083D082120AC9120A5A
:100AC000C9120AC9120AC9E473E493A3C583C5F025
:100AD000C583C8C582C8F0A3C583C5F0C583C8C592
:100AE00082C822EC8EF0A4CCC5F0CCCDF8EFA4CE19
:100AF000C5F02DFDE43CFCE8A42EC8C5F03DFDE4A6
:100B00003CFCEFA4FFE5F028FEE43DFDE43CFC22C4
:100B1000EF4E6012EF60010EEDBB010B89828A83FC
:100B2000F0A3DFFCDEFA2289F05007F709DFFCA909
:100B3000F022BBFEFCF309DFFCA9F022BC000BBED7
:100B40000029EF8DF084FFADF022E4CCF875F008B9
:100B5000EF2FFFEE33FEEC33FCEE9DEC984005FCEE
:100B6000EE9DFE0FD5F0E9E4CEFD22EDF8F5F0EEB6
:100B70008420D21CFEADF075F008EF2FFFED33FDA1
:100B80004007985006D5F0F222C398FD0FD5F0EA41
:100B900022E6FC08E6FD08E6FE08E6FF22E0FCA3EC
:100BA000E0FDA3E0FEA3E0FF22E2FC08E2FD08E294
:100BB000FE08E2FF22E493FC740193FD740293FEAD
:100BC000740393FF22E6FB08E6F908E6FA08E6CB91
:100BD000F822E0F8A3E0F9A3E0FAA3E0FB22E2FBAD
:100BE00008E2F908E2FA08E2CBF822E493F874018B
:100BF00093F9740293FA740393FB22ECF608EDF672
:100C000008EEF608EFF622120FD11210729001C80A
:100C1000120FD4F912088CFDACF0D39FEC9E403635
:100C2000120FD1121146FFEC95F0FED3EF9430EE87
:100C30009475400C9002537475F0A37430F0800FDB
:100C40001210739001C8120FD412119B1210F9E404
:100C5000900219020CCD9001C8120FD4121072121A
:100C60000FD1F912088CFDACF0C39FFFEC9EFED3B0
:100C7000EF9410EE9427400C9002537427F0A37465
:100C800010F080149001C8120FD4121146FEEC959A
:100C9000F0900253F0A3CEF0900253E0FFA3E09057
:100CA0000219CFF0A3EFF0300018D3E0942C90029B
:100CB00019E09401401390021B7427F0A37410F004
:100CC0008007E490021BF0A3F0E4900253F0A3F03D
:100CD0009001E9E0605412108ED39400EE64809489
:100CE00080401A9001C2E0FCA3E0FDD3EF9DEE9C92
:100CF000400B90022CE4F0A37464F0801FD39002A8
:100D00002DE0940090022CE0940040109001CB1252
:100D10000FD4F912088CFFE5F01210F9D20B9002F3
:100D200032740FF0A374A0F0800C1211147B007ABF
:100D3000007930121014D3900254E09400900253C2
:100D4000E0648094805003020F8BE0F9A3E0FF90F1
:100D500001CB120FD412108812108E1211E7E47B0F
:100D6000B87A88F9F8C31209F3500A9002537488CC
:100D7000F0A374B8F0D390022FE0940090022EE01C
:100D80009400500790003AE0B4201D12108EC394D6
:100D900096EE648094805010EF9400EE648094800E
:100DA000404E7C007D0A80103000459001E9E070E3
:100DB0000C12108E7C027DBC1210F580339001C2A3
:100DC000E0FCA3E0FD12108EC39DEE9C50227C023D
:100DD0007DBC1210F51211147E007F1F7D007B0078
:100DE0007A007930120B10121178120FD412108879
:100DF0009001E9E07003020F69900230E07002A3F5
:100E0000E06003020F6912108E1211E7E5332FF52F
:100E100033E5323EF532E5313DF531E5303CF53034
:100E20000535E53570020534C3E53994D0E53894CD
:100E3000075003020EF8AE34AF35CBEFCB12110DD5
:100E4000AF33AE32AD31AC30120961900255EEF0E5
:100E5000A3EFF0C3E5379FFFE5369EFE122BEA9025
:100E60000257EEF0A3EFF0D39464EE94005006E541
:100E7000374536700D900255E0F536A3E0F53702A0
:100E80000EE7D3900256E09537900255E095364034
:100E90002812111F400474148018D3EF943CEE9470
:100EA000004004740A800BD3EF9428EE940040377E
:100EB00074052537F537E4802A12111F400774ECBA
:100EC0001211EE801ED3EF943CEE9400400774F6AE
:100ED0001211EE800ED3EF9428EE9400400974FBBB
:100EE0001211EE3536F536E4F533F532F531F530DD
:100EF000F534F535F538F539D3E5379400E5369412
:100F0000004028120FB5900202EEF0A3EFF0C312DA
:100F10000FB51211DD50081211A6E4F53A800CE568
:100F20003AC3940750051211A6053AE5DB20E24AC0
:100F30009001D4120FD41210727C007D0F120AE3BC
:100F4000C8ECC8C9EDC9CAEECACBEFCB12108E12DD
:100F500011E7EB121032E47B10FAF9F812096190F4
:100F600001D4120FD4F9EE800CE5DB20E20C121153
:100F700078120FD4C98FF01208B79001D4120FD491
:100F8000F912088C24A8FFE5F0801D9001CB120F08
:100F9000D41210EE9001D4120FD41210EE9002541D
:100FA000E024A8FF900253E03461F99001D1120FC0
:100FB000D412108822900254E09537FF900253E03B
:100FC0009536FE122BEA229001EBA3A3E0F9A3E0F1
:100FD000FF9001CEE0FBA3E0FAA3E022E4FAF9F8E7
:100FE000E0FCA3E0FDA3E0FEA3E0FF22E47F607E3F
:100FF000EAFDFCE0F8A3E0F9A3E0FAA3E022F07E2A
:10100000007F077D007B007A007953120B107BFE76
:101010007A0079007E007F1F7D00020B10E4FFFE46
:10102000FDFCE2FB08E2F908E2FA08E2CBF8C302B1
:101030000A092FFFEA3EFEE93DFDE83CFC22E2FC06
:1010400008E2FD08E2FE08E2FF020A9ACBEFCBCAF3
:10105000EECAC9EDC9C8ECC8E0FCA3E0FDA3E0FE00
:10106000A3E0C39BFFEE9AFEED99FDEC98FCA30272
:101070000A9AF912088CFFAEF022F043AB0A5389AA
:10108000F55395F55396F522C98FF00208B79002F3
:1010900053E0FEA3E0FF22A3F0A37401F0A322F02B
:1010A0009002287402F0A37458F0227F087A017924
:1010B000EB7E007D007B01020B10902E127D0AE07A
:1010C000FEA3E0FF7C0002082EE50825E0242AF8B4
:1010D000E622900251A3A3E0F9A3E0FF9001C82209
:1010E000E2FC08E2FD08E2FE08E2FF020A9AF9E4E7
:1010F000F5F00208B7120840EE900253F0A3EFF0AB
:101100002290003AE0642022E0FEA3E0FBCAEECA8F
:10111000E4F9F8229002307403F0A374E8F022900E
:101120000257E0FEA3E0FFD39450EE940022758DA9
:1011300020438D20758D8043A808D2AF229001C630
:10114000E0FCA3E0FD22F912088CFFC3ED9F22FE14
:10115000ED39FDEC38FC020A9A90021FE4F0A3740A
:10116000C8F02225E02408F582E43402F583E02269
:10117000902E12E0FEA3E022900253E0F9A3E0FFDC
:101180009001D422D3900220E09F90021FE09E2283
:1011900025E0242AF8A60D08A60E22F912088CC311
:1011A0009FFFE5F09E22900253E536F0A3E537F06D
:1011B00022E490022EF0A3F0229001C2E4F0A37486
:1011C00096F022F9746175F0A80208B7900059747E
:1011D00010F022E4F50CF50BF50AF50922C3EF94A3
:1011E00064EE6480948022EE3395E0FDFC22253786
:1011F000F53774FF22758B11758A3053A8F722C317
:10120000E5529564E551956322208A0302144790C4
:101210000228E07002A3E06003021447900226E077
:101220007002A3E06003021447900204E07002A37E
:10123000E060030214471211016003021447900199
:10124000E9E0703A9001DD120FD41210729001CBD8
:10125000120FD4F912088CD39FE5F09E40030214BC
:10126000471210ABE4900210F0A3F01211B29002FA
:101270002CF0A3F0900236F0A3F0F56380037563C1
:101280000075640AE4F5B212297A900214E0F54F71
:10129000A3E0F550C209E4F55DF55CF55BF55A1283
:1012A000112E758B02758EC8200524121101701F36
:1012B000200C1CE5DB20E217758AA4200C0DE5DB71
:1012C00020E2087587030000008006D2098002D260
:1012D000091211F5D3900227E09490900226E09431
:1012E00001400EA3E02470F0900226E034FEF0806E
:1012F00007E4900226F0A3F0D3900233E09490909C
:101300000232E09401400EA3E02470F0900232E03B
:1013100034FEF08007E4900232F0A3F012297A1232
:10132000228A856865856966856824856925902E89
:1013300023E4F043890A1210815380F54389029017
:101340000200E524F0A3E525F0C3E5509525FFE56F
:101350004F9524FE122BEA8E518F521211FF40033B
:10136000021419AE24AF257C007D02120AE390021C
:1013700051120A9A900251120FECFBD3120A094043
:101380000A900251120AB20000EA609001C8120FDE
:10139000D41210727C007D09120AE3900251120FE0
:1013A000F3121032E47B0AFAF9F812096190025143
:1013B000120A9A9001E9E0702CAE24AF25FCFDFBE7
:1013C0007A00795A900272740AF0121E428E4F8F80
:1013D00050900251120FCA1210881210D2120FD45C
:1013E00012108880341210D2120FD4121088120FEB
:1013F000D1121072E4FCFD900251120FF3FBD312D4
:101400000A094025120FD11210729001C8120FD490
:1014100012119BFE121184501020090D1211FF5061
:1014200008121101700302129F900218E004120FBB
:10143000FEE49001FCF0A3F0A3F0A3F09001EA0415
:10144000F090022A12115C22900210E0FEA3E0FF4D
:10145000C39404EE9400502A12113DEF25E0FFEEF4
:1014600033FE74082FF58274023EF583ECF0A3ED91
:10147000F0900211E004F07006900210E004F00217
:1014800015D190025B7401F090025BE0FF121163D2
:10149000FCA3E0FDEF25E02406F582E43402F583A9
:1014A000ECF0A3EDF090025BE004F0E0B404D9901E
:1014B00001E9E07003021563120FD11210721211CC
:1014C0003DD39FEC9E5003021561ED9FFFEC9EFE05
:1014D000D3EF94F4EE94015003021561A3120FD4DC
:1014E000121146FFEC95F0FE90025CF0A3EFF012B3
:1014F0002BEA1211DD506AE490025EF0A3F0900234
:101500005CE0FEA3E0FF122BEAD3EF9428EE6480A8
:1015100094804025D390025DE0940090025CE064EA
:1015200080948090025E4008E4F0A37405F080107F
:1015300074FFF0A374FBF08007E490025EF0A3F068
:101540009001C8120FD4F912088CFF90025FE02FAF
:10155000FE90025EE035F090020EF0A3CEF0021590
:10156000D1805F9001C8120FD4F912088CFF1211BC
:101570003DC3EF9DFFE5F09CFE122BEAC3EF9428DC
:10158000EE64809480503B120FD1F912088CFFC397
:101590009001C7E09FFF9001C6E095F0FE122BEA94
:1015A000C3EF9414EE6480948050059001CE8003C4
:1015B0009001C8120FD4F912088CFF90020EE5F0CA
:1015C000800B9001C6E0FFA3E090020ECFF0A3EFE6
:1015D000F0900257120AB200000000E490025BF0A3
:1015E00090025BE0FFD3900211E09F900210E09424
:1015F000004026900257120FF3FBA3E0121163FE86
:10160000A3E0FFE4FCFDEB2FFFEA3E90025712112E
:101610004F90025BE004F080C7900257120FE0EE9B
:10162000C0E0EFC0E0900210121108D0E0FFD0E05F
:10163000FE120961900257120A9A900257A3120FE4
:10164000E522C0E0C083C082C0D0E8C0E0D2AFE5F0
:101650006D2401F56DE4356CF56CE4356BF56BE4E8
:10166000356AF56AD3900227E09400900226E09450
:1016700000400CA3E024FFF0900226E034FFF0D3FA
:10168000900229E09400900228E09400400CA3E02E
:1016900024FFF0900228E034FFF0D390022BE09476
:1016A0000090022AE09400400CA3E024FFF0900296
:1016B0002AE034FFF0D390022DE0940090022CE059
:1016C0009400400CA3E024FFF090022CE034FFF0E3
:1016D000D390022FE0940090022EE09400400CA3DF
:1016E000E024FFF090022EE034FFF0D3900237E0C8
:1016F0009400900236E09400400CA3E024FFF090A8
:101700000236E034FFF0D3900231E09400900230D2
:10171000E09400400CA3E024FFF0900230E034FF9E
:10172000F0C37809E294E818E29403500A08E2242E
:1017300001F218E23400F2C3E53994D0E538940799
:1017400050080539E53970020538D3900205E09458
:1017500001900204E09400400CA3E024FFF090020A
:1017600004E034FFF0D3900233E09400900232E0C2
:101770009400400CA3E024FFF0900232E034FFF02C
:10178000D390021CE0940090021BE09400400CA354
:10179000E024FFF090021BE034FFF0D3900222E03F
:1017A0009401900221E09400400CA3E024FFF0900B
:1017B0000221E034FFF0D3900241E0940090024017
:1017C000E09400400CA3E024FFF0900240E034FFDE
:1017D000F0D0E0F8D0D0D082D083D0E03290025860
:1017E000EFF0902E227401F01228687402F0A3E446
:1017F000F0900259F0900259E0FFC3940C400302AC
:1018000018E7E47E01C8EFC8088006CEA2E713CE31
:1018100013D8F8FF90025AEEF0A3EFF04E70079045
:10182000025AF0A304F0902E207409F0902E20E0CC
:1018300030E2F9900258E0FF75F002A4240012286B
:1018400072E0FCA3E0D394FFEC9407404175F002F2
:10185000EF12286FE0FEA3E0FF90025AE0FCA3E045
:10186000FDEF2DFFEE3CFEC3EF94FFEE94039002DC
:1018700058E075F002500B12286FEC8DF0120876CC
:10188000805412286F7403F0A374FFF08048900214
:1018900058E0FF12286CE0FCA3E0FD90025AE0FA49
:1018A000A3E0FBD3ED9BEC9A402575F002EF1228E4
:1018B0006FC083C082C3A3E09BFF0582D58202155F
:1018C000831582E09AD082D083F0A3EFF0800712D4
:1018D0002868E4F0A3F0902E20E4F0438D209002DD
:1018E00059E004F00217F5221211D3F513F514850F
:1018F0002A0F852B10852A11852B12F5081210C985
:10190000FE08E6FFD3E5129FE5119E40078E118F7A
:1019100012850814C3E5109FE50F9E50078E0F8FA8
:10192000108508130508E508B402D2E4F50DF50E9C
:10193000F508E51465086032E5136508602CE50ECE
:10194000450D700B1210C9F50D08E6F50E801B123F
:1019500010C9FE08E6250EFFE50D3EFEEF2401FF4F
:10196000E43EC313F50DEF13F50E0508E508B402C8
:10197000C1900214E50DF0A3E50EF0C3E51494FF49
:101980007480947F5005E514121190C3E51394FF01
:101990007480947F5005E5131211901211D3F5084D
:1019A0001210C9FE08E6FFE4FCFDE50C2FF50CE57E
:1019B0000B3EF50BED350AF50AEC3509F50905087E
:1019C000E508B402DBE47F607EEAFDFCAB0CAA0B09
:1019D000A90AA809D3120A09400BE4750C60750B1B
:1019E000EAF50AF509AE0BAF0C229001E9E06006BA
:1019F0001210AB021ADA9001EB120FF3FBE9C0E010
:101A0000EAC0E0EBC0E09001C8120FD4F912088CD4
:101A1000FFE4FCFDD0E0FBD0E0FAD0E0F9EB2FFFD3
:101A2000EA35F09001EB12114F9001F0E004F070F4
:101A3000069001EFE004F090022AE07002A3E0605B
:101A400003021AE49001EB120FE0EEC0E0EFC0E0F9
:101A5000A3121108D0E0FFD0E0FE1209619001EB63
:101A6000120A9A120FD1F912088C2432FFE435F0D1
:101A7000FEE4FCFD9001EB120FF3FBD3120A0940C8
:101A800039900226E07002A3E0702F200B2C900109
:101A9000F2E004F070069001F1E004F0D39001F25E
:101AA000E094059001F1E09400401E120FC712105F
:101AB00088E49001F1F0A3F0800F120FC712108894
:101AC000E49001F1F0A3F0C20B9001EB120AB20016
:101AD000000000E49001EFF0A3F090022A7407F0F8
:101AE000A374D0F022900142E0FEA3E0FFC3900176
:101AF0002BE09FFF90012AE09EFE122BEAD3EF9489
:101B00000AEE648094804020900122120AB2000004
:101B10000000E4900126F0A3F0900142E0FFA3E072
:101B200090012ACFF0A3EFF0900122122616900127
:101B3000421225D0900122120A9A900127E004F067
:101B40007006900126E004F0900126E0FEA3E0FF7D
:101B5000D3940AEE94004031CBEFCBCAEECAE4F93D
:101B6000F890012212260A120961900128EEF0A3D2
:101B7000EFF0A3EEF0A3EFF0900122120AB2000002
:101B80000000E4900126F0A3F0D3900129E0940036
:101B9000900128E09400403090012CE0FEA3E0FF8B
:101BA0007C007D03120AE3C8ECC8C9EDC9CAEECABD
:101BB000CBEFCB9001281225D0E47B04FAF9F81280
:101BC000096190012CEE800B900142E0FFA3E090B0
:101BD000012CCFF0A3EFF0227E007FFF7D007B0180
:101BE0007A007923120B109002767400F0A374230C
:101BF000F0902DE0E493FF900276E0FCA3E0FDF589
:101C0000828C83A3EFF0900021E0FFED24041228E2
:101C10007B900020E0FFED240512287B900022E05D
:101C2000FFED240612287B902DE2E493FFED2412B1
:101C300012287B902DE3E493FFED241412287BE41B
:101C4000FF75F002EFA42401F582E5F0342EF58350
:101C5000E493FE122895EEF0122895E0FE75F0024E
:101C6000EFA42400F582E5F0342EF583E4932420DC
:101C7000F582E4342EF583EEF00FEFB411C3902F0C
:101C800056E0900077F0902F56E0900089F0900198
:101C90001E7401F090011DF09000597410F0900036
:101CA0003AF0900047F0A37420F09002267407F0F9
:101CB000A374D0F02290025B120A9A90025B120F7A
:101CC000E07BFE7A00791B9002727403F0121E42D0
:101CD000E4FCFD90025B120A9AE4FFFEFDFC78171B
:101CE000121022600CE4FFFEFDFC7813121022702B
:101CF0002090025B120FE07817120AA6E47F20FE04
:101D0000FDFC90025B120FF3FB1208D67813120A47
:101D1000A6781790025F1210E078139002631210F9
:101D2000E0900263120FE07804120A1A9002631224
:101D3000104C90025F120FE090025B120FF3121032
:101D400032900267120FF3121032900263120A9A55
:101D500090025B120FE07817120AA6900263120F2E
:101D6000E07813120AA67B20900263120FDC12099E
:101D700061900267120A9A900267A3120FE52290FF
:101D80000259120A9A780F12101D6007780B121070
:101D90001D7020900259120FE0780F120AA6E47FFE
:101DA00010FEFDFC900259120FF3FB1208D6780BBF
:101DB000120AA6780F90025D12103E780B90026115
:101DC00012103E900261120FE07803120A1A90027C
:101DD0006112104C90025D120FE0900259120FF345
:101DE000121032900265120FF3121032900261123B
:101DF0000A9A900259120FE0780F120AA690026117
:101E0000120FE0780B120AA67B10900261120FDC11
:101E1000120961900265120A9A900265120FECFB9A
:101E2000D3120A09400A900265120AB20000EA6061
:101E3000900265A3A3E0FFA3E0900200CFF0A3EF20
:101E4000F02290026B120A9A90026FEBF0A3EAF074
:101E5000A3E9F090026B120FE07804120A2D9002B1
:101E60006B120A9A120A40E4FBFAF9F8C3120A0943
:101E7000701990026B120FE0A3120FD4F9120A60CE
:101E800090026B120FE07804020A1A900272E024AA
:101E9000FFFFE434FFFEE4FCFD90026F120FD4F963
:101EA000120A7A1208D690026B120FF3121032EF58
:101EB000C0E0900272E0FBE4FAF9F8D0E0FF12090A
:101EC000618F118E108D0F8C0E90026F120FD4F94E
:101ED000120A60AF11AE10AD0FAC0E7804120A1AE0
:101EE0008F118E108D0F8C0E22D3900227E094005C
:101EF000900226E094004003021F8E30001E9002E4
:101F00001BE07002A3E090021F7405F0A374DCF0E4
:101F10009001C27405F0A37414F0800612115912D6
:101F200011B99001CB120FD4121072121184401308
:101F30009001E9E0601ED39001C3E09F9001C2E0F0
:101F40009E501190022EE07002A3E0702A9001E9E9
:101F500004F0802390003AE0B420051211B180090A
:101F600090022EE4F0A37464F0E49001E9F0900292
:101F70002CF0A3F01211CC9001E9E0601190004721
:101F8000E0900059B410047410F0227420F0227F05
:101F9000597A0179C61210B19001C87401F0A37486
:101FA00000F074631210977400F074651210977447
:101FB00000F0A374671210987400F0A3745112100B
:101FC000987400F0A3744D1210987400F0A3744B31
:101FD000F09001E67401F0A37400F0A3743BF0905C
:101FE00001DA7401F0A37400F0A374551210987410
:101FF00000F0A374491210987400F0A37457F01203
:1020000011599001DA120FD4F9E475F0C81208B72B
:102010009001DD120FD4F9E475F0641208B71211C3
:10202000B99001E0120FD4F9E475F0960208B7C038
:10203000E0C083C082C0D075D018D2AFE5DB30E4F9
:1020400022D20CC208E5DB30E114122A5FE0F5DF92
:10205000EFB40708208A05122A47E4F08049C20637
:102060000220C1E5DB30E517D205300804C2088044
:1020700002C20C9002407407F0A374D0F08042C2F8
:1020800008E5DB30E126E5DB30E036122A5FE0F5DB
:10209000DFEFB4070A208A0F122A47E4F08008789D
:1020A00015E6B41902D207781506801578152006B2
:1020B00008A6DFD206D2088008E6122A63E5DFF020
:1020C0000675DBFFD0D0D082D083D0E032900253AF
:1020D000EEF0A3EF120FFE900253E07002A3E06057
:1020E00003122166E4900210F0A3F07F021229AEE1
:1020F0001210A0A37407F0A374D0F09001C6E0F909
:10210000A3E0FFA3120FD41210889001CB120FD4BA
:102110001210EE9001D1120FD41211C39001D412FB
:102120000FD41210EE9001D7120FD41211C3121156
:10213000CCE49001E9F09001EB120AB2000000003B
:10214000E49001EFF0A3F0A3F0A3F09001C6120F0A
:10215000CC121088E49001EAF0900236F0A3F090DF
:102160000232F0A3F022E4F5677F01122B781211FE
:1021700070C394FFEE940150061211704E700875F2
:1021800067017F01122B7812117024E0FFEE34FCFE
:10219000900255F0A3EF12107A12297A122B1D909B
:1021A0002E227401F0902E207409F0902E20E03041
:1021B000E2F9902E027D031210BF8E288F291D1286
:1021C0000AE38F628E618D608C5F902E20E4F04375
:1021D000890A1210815380F5902E23F09001C5E0FA
:1021E000900040F01210BAEF244CFFEE3404F99046
:1021F00001E6120FD4C98FF00208B7787FE4F6D851
:10220000FD75816D0222450200000228D8E493A3E7
:10221000F8E493A34003F68001F208DFF48029E498
:1022200093A3F85407240CC8C333C4540F4420C8E4
:10223000834004F456800146F6DFE4800B0102047B
:102240000810204080902319E47E019360BCA3FF16
:10225000543F30E509541FFEE493A360010ECF54B0
:10226000C025E060A840B8E493A3FAE493A3F8E49F
:1022700093A3C8C582C8CAC583CAF0A3C8C582C80B
:10228000CAC583CADFE9DEE780BEE4900259F0A345
:10229000F0F508F509F50AF50BF50CF50D12107BB4
:1022A000F0E4F508F509900259F0122B1D902E204C
:1022B0007409F0902E20E030E2F9902E02E0F50C47
:1022C000A3E0F50DAE0CFFE4FCFD121CB5EF2509F3
:1022D000F509EE3508F508902E20E4F0900259E05B
:1022E00004F0E0C3940340C2E509250BF50BE508B3
:1022F000350AF50A90025AE004F0E0C3940140A1C7
:10230000850A68850B69902E23E4F0902E20F04317
:10231000890A1210815380F5224102480041024986
:102320000041024F004102450041024D004202219E
:1023300003E841025000C101C10341024E004102C5
:102340004400C102C100C104C1060115004202736C
:102350000000C105C108C107410275104101C1005B
:102360004101C510C10BC10A016700022800000429
:102370005F00000000015E004101C41041012F0018
:10238000046A0000000041012E004101B200420138
:102390004200004401B30000000042012C00004153
:1023A00001B700C10C00900244E014601B146043AC
:1023B0002402705D90024EE0B4010A90024412249F
:1023C00012D204D200C202227F021228A0EF6007BC
:1023D0007F02122BF6C20490024EE0703490024449
:1023E0007402F0D202C204C2007F03122BF67F03F4
:1023F000022AA37F031228A0EF60167F03122BF698
:1024000090024EE09002447003F08003122412C246
:1024100002227401F07F02122BF67F02122AA322FD
:1024200012228AE529240CFFE52834FEFED3EF951D
:1024300069EE95684015900204E07002A3E0701206
:1024400090020404F0A374F4F08007E4900204F016
:10245000A3F09001FEE568F0A3E569F0FFAE689097
:1024600001FAEEF0A3EFF0E4FCFD121D7F900200F4
:10247000E0F52EA3E0F52F7F01EF1210CBFC08E66C
:10248000FDEF25E02428F8C6ECC608C6EDC60FEF20
:10249000B403E622E4F5B275B6FF75B7FF75B2A2D4
:1024A00043B201122BD09001B77401F0E5A830E2DD
:1024B000030080F890012EE0FFE4FCFDFE122600F0
:1024C00012260A7808120A2D1226001226169001EA
:1024D000B2E0FFEB4FFFEAFEE9FDE8FCA3122603A2
:1024E000A3A3E0FFA3E0900142CFF0A3EFF0538B52
:1024F000EF53A8FBE4F5B2122B94021AE5900221E7
:10250000E07004A3E064017011900250E07004D206
:102510008A04F0E4900221F0A3F0900059E0FC90CE
:1025200001C4E06C6039900059E0FE9001C4F09065
:10253000002AE090024DF0540FF0EEB42005E04484
:1025400020800AECB4100B90024DE04410F0900093
:102550002AF0C28AE4900250F09002211211172250
:10256000200A06200203300412300A067F017E0092
:102570008003E4FFFE1220CDC20A22900236E070F2
:1025800002A3E06005121101703420000312282517
:102590007F011229AE121448900251EEF0A3EFF021
:1025A0007B017A02795112278D9002511210D712B5
:1025B0000FD4121088120C07121EE91219EA122405
:1025C000FD22CBEFCB74B82BF582E43401F58322E6
:1025D000E0FEA3E0FFE4FCFDEB2FFFEA3EFEED3959
:1025E000FDEC38FC22FEEB25E02430F582E43401DA
:1025F000F58322EB25E0240BF582E4342BF58322CE
:102600009001B3120A9A9001B322E0FCA3E0FDA36B
:10261000E0FEA3E0FF22E0F8A3E0F9A3E0FAA3E0E4
:10262000FB229002517408F0A3E4F0A3743FF0A3DE
:1026300074DFF0E4FDFCF9758A10538AEF00900214
:1026400051E0FEA3E02DF582EE3CF583E493FF69B3
:10265000F90DBD00010CBC37E5BDDFE2900253125D
:102660002A6DE493699002767009122A6DA37404AE
:10267000F08006122A6DA3E4F0758A30538AEF00C9
:1026800022308A59900226E07002A3E0704F900237
:1026900004E07002A3E07045121101604090024016
:1026A000E0FEA3E0FFD39400EE9400503012112E10
:1026B000E4F58B758E10200521200C1EE5DB20E251
:1026C00019EF4E7015758AA4200C0FE5DB20E20A85
:1026D000EF4E70067587030000001211F5221228D4
:1026E0008DF5828E83A3E0B4AA0312262212288DD0
:1026F000FF122884E0B41008EF122884E4F0D20A14
:1027000012288DFF241B122886E0700DEF241C1266
:102710002886E0B410031227DA12288D2413122819
:1027200086E0FFB4100690024E7401F0EFB420056D
:10273000E490024EF022900225E024FE6013146023
:1027400023146027240370449002257402F01208B9
:10275000037F017E001220CD9002257403F0E490E7
:102760000245F0229002257404F0221223A61229B9
:102770000F1223A6900204E07004A3E06401700C21
:10278000900204F0A3F09002257402F0229002530C
:10279000EBF0A3EAF0A3E9F0900228E07002A3E0D6
:1027A00070379001EAE06031E49001EA12109F90E6
:1027B00002567401F07F011229AE121448900253A0
:1027C000120FD4F9EE8FF01208B7900256E004F021
:1027D000E0C3940240DF1211B122758A10538AEFD0
:1027E00000122B40E4F5F275F30875EEFF75EF3F2C
:1027F00075EA81F5F675EB0700E5EC30E7FBE4F5EB
:10280000EC900276E0FEA3E0FF241B122A58E5F3C9
:10281000F0EF241C122A58E5F2F075EB30758A307F
:10282000538AEF002230073FC207902E12E0FFA329
:10283000E0900253CFF0A3EFF0E4FF122B781210D8
:10284000BAEF244CFFEE3404FE9001E6120FD4F9E7
:10285000EE8FF01208B7900253E0FFA3E0902E1223
:10286000CFF0A3EF12109F22900258E075F002A45F
:102870002410F582E5F0342EF58322F582E43CF550
:1028800083EFF022241AF582E43EF583229002764B
:10289000E0FEA3E02274732FF582E43400F5832276
:1028A0001225C2E0602FE56DFFE56C1225E5E0FC26
:1028B000A3E0FDD39FEC9E501CC3EF9DFFEE9CFE5A
:1028C0001225F3C37401939FE4939E40081225C51B
:1028D000E4F07F01227F0022122BDD53A87F122912
:1028E00045122BC3122ACE122BAE43A88012249479
:1028F00090011EE0600B9002257401F0E490011E2F
:10290000F0122B5C1226DE12273612249480E190FE
:102910000048E06420702890003AE0B4201490024F
:102920003FE070031210A090023F7401F0121209F0
:102930008008E490023FF012268112256080031285
:102940002A76022B94758A30538AEFE4F58F900033
:10295000217411F09000207422F09000227433F062
:10296000E4F5AB75AC0C7589FF75913CF595F59266
:10297000D28A90025004F0D20D22902E23E4F0FF70
:1029800074732FF582E43400F583E0FE75F002EFF6
:10299000A42400F582E5F0342EF583E4932420F599
:1029A00082E4342EF583EEF00FEFB411D3229002BF
:1029B00057EFF012297AE4900258F0900257E0FFA6
:1029C000A3E0C39F500B122420900258E004F08033
:1029D000EA902E20E4F01218E89001C6EEF0A3EF82
:1029E000F022E4FEE4FFEF75F003A42444F582E452
:1029F0003401F583E5822EF582E43583F583E4F036
:102A00000FEFB40AE10EEEB403DA7F099001B8E4E7
:102A1000F0A3DFFC22C0E0C083C0829001B7E06079
:102A20000DE4F0538B7F758B11438B088012538B11
:102A30007F53A8FBE5B590012EF0E5B49001B2F00C
:102A4000D082D083D0E032D28A9002507401F090CC
:102A50000276E0FEA3E02407F582E43EF5832278C7
:102A600015E6FF2423F582E43400F58322E0FEA37B
:102A7000E0F5828E8322E4F5B2F5BA758D20438DA0
:102A800020538D7F53AAF7F58BE5DB20E211200C54
:102A90000EE4F58A758703000000758A30D20A7546
:102AA0008B11221225C2E060037F01221225C5741A
:102AB00001F01225F3E493FE740193FFEF256DFFFF
:102AC000EE356C1225E5EEF0A3EFF07F00229002C8
:102AD00076E0FFA3E0A3CFF0A3EFF0E4F5DA75DA38
:102AE0004043DA2075D74075DA5875D90143A802FA
:102AF00075B80475F8042201F40028002801F400D8
:102B00009603E801F403E81770006403E80032025A
:102B1000580258012C01F403E8271000C8E567901B
:102B20002E21B401057411F080037491F0902E24CD
:102B30007401F0902E277414F0902E237402F0226A
:102B400074AA7583F5758255A574557583FA7582D7
:102B5000AAA574A57583F5758255A522E4FF3005F5
:102B600016900276E0FCA3E0F5828C83E0FE54F040
:102B7000FFEE540FF0C20522900257EF12107A12A6
:102B8000297A122B1D7F011217DD43890A12108149
:102B90005380F522E5B230E005E5A820E40F75B2D8
:102BA0009275B67CE4F5B743B20143A810227E00CB
:102BB0007F0A7D007B017A017922120B1012081620
:102BC0000229E2121BD8121F8F9002257401F022F5
:102BD000538B7F758B10438B0843A804225391FCC1
:102BE00043920390027A7440F022EE30E707C3E488
:102BF0009FFFE49EFE2274B82F1225C8E4F0220045
:102C000000000000000000000000000000000000C4
:102C100000000000000000000000000000000000B4
:102C200000000000000000000000000000000000A4
:102C30000000000000000000000000000000000094
:102C40000000000000000000000000000000000084
:102C50000000000000000000000000000000000074
:102C60000000000000000000000000000000000064
:102C70000000000000000000000000000000000054
:102C80000000000000000000000000000000000044
:102C90000000000000000000000000000000000034
:102CA0000000000000000000000000000000000024
:102CB0000000000000000000000000000000000014
:102CC0000000000000000000000000000000000004
:102CD00000000000000000000000000000000000F4
:102CE00000000000000000000000000000000000E4
:102CF00000000000000000000000000000000000D4
:102D000000000000000000000000000000000000C3
:102D100000000000000000000000000000000000B3
:102D200000000000000000000000000000000000A3
:102D30000000000000000000000000000000000093
:102D40000000000000000000000000000000000083
:102D50000000000000000000000000000000000073
:102D60000000000000000000000000000000000063
:102D70000000000000000000000000000000000053
:102D80000000000000000000000000000000000043
:102D90000000000000000000000000000000000033
:102DA0000000000000000000000000000000000023
:102DB0000000000000000000000000000000000013
:102DC0000000000000000000000000000000000003
:102DD00000000000000000000000000000000000F3
:102DE0000401AB37000000000000000000000000FC
:102DF00000000000000000000000000000000000D3
:102E00000191020107140AB00BB60CFF090008FF7C
:102E10000DF70E060F040401110612061307141015
:102E20001010000000000000000000000000000082
:102E30000000000000000000000000000000000092
:102E40000000000000000000000000000000000082
:102E50000000000000000000000000000000000072
:102E60000000000000000000000000000000000062
:103FD000000000000000000000000000000000A43D
:103FE00000000000000000000000000000000000D1
:103FF00000000000000000000000000000000000C1
:00000001FF
